:020000040000FA
:100000000000000000000000000000008316F73030
:1000100081008312073099008501E5298207393470
:10002000A60B102800340A30A7000000A60B1528E4
:10003000A70B152800346030A7001020A70B1D283F
:1000400000343230A8001320A80B23280034831674
:10005000FF308500831221200034A901A915552005
:10006000A9156420A9157520A9158620A915972022
:10007000A915A820A915B920A915CA20A915DB2002
:10008000A915EC20A915FD20A9150E21A9151F21E0
:10009000A9153021A9154121A9155221A9156321BE
:1000A000A9157421A915852100348316CD3085004A
:1000B00083122630850013208316FF3085008312BB
:1000C0001320A90B552800348316E93085008312CC
:1000D0001030850013208316DD3085008312023036
:1000E00085001320A90B642800348316CD308500C9
:1000F00083120030850013208316ED3085008312B3
:10010000123085001320A90B752800348316DF30C8
:10011000850083121030850013208316E13085009E
:100120008312063085001320A90B8628003483161D
:10013000E930850083120430850013208316CF3008
:1001400085008312103085001320A90B97280034F6
:100150008316E93085008312003085001320831652
:10016000CB3085008312143085001320A90BA828FA
:1001700000348316ED308500831201308500132092
:100180008316FD3085008312033085001320A90BF0
:10019000B92800348316C9308500831200308500E9
:1001A00013208316E9308500831216308500132052
:1001B000A90BCA2800348316E93085008312043065
:1001C000850013208316CD30850083121230850000
:1001D0001320A90BDB2800348316E8308500831236
:1001E0000130850013208316E83085008312173014
:1001F00085001320A90BEC2800348316FC30850001
:1002000083122730850013208316EE308500831279
:10021000013085001320A90BFD2800348316E83037
:10022000850083121130850013208316DC30850091
:100230008312033085001320A90B0E290034831686
:10024000CC30850083120130850013208316EC30FA
:1002500085008312133085001320A90B1F29003459
:100260008316CA308500831205308500132083165B
:10027000FC3085008312033085001320A90B302940
:1002800000348316E8308500831205308500132082
:100290008316CE3085008312113085001320A90B00
:1002A000412900348316E83085008312013085002F
:1002B00013208316CA308500831215308500132061
:1002C000A90B522900348316EC30850083120130CB
:1002D000850013208316FC308500831203308500CF
:1002E0001320A90B632900348316C83085008312BC
:1002F0000130850013208316E0308500831217300B
:1003000085001320A90B742900348316E83085007A
:1003100083120530850013208316CC3085008312AC
:10032000133085001320A90B852900348316EB3088
:10033000850083120030850013208316E930850084
:100340008312163085001320A90B962900348316DA
:10035000FB30850083120030850013208316EB30BC
:1003600085008312143085001320A90BA7290034BF
:100370008316E93085008312003085001320831630
:10038000E93085008312163085001320A90BB829A7
:1003900000348316F9308500831200308500132065
:1003A0008316CB3085008312143085001320A90BEF
:1003B000C92900341030A3008316FF308500831252
:1003C00010201020A30BDC290034A9012D20A91531
:1003D00085218519E7291030A100A9148521DA218A
:1003E000A10BED29A9158521851DF22927201F3094
:1003F000A400A91574211020851D012AA40BF92938
:10040000B32B1030A1002108A300A9147421DA2114
:10041000A10B032AA9157421851D0A2A27201F3044
:10042000A400A91563211020851D192AA40B112AE7
:10043000B82B1030A1002108A300A9146321DA21F0
:10044000A10B1B2AA9156321851D222A27201F30F5
:10045000A400A91552211020851D312AA40B292A98
:10046000BA2B1030A1002108A300A9145221DA21CF
:10047000A10B332AA9155221851D3A2A27201F30A6
:10048000A400A91541211020851D492AA40B412A49
:10049000C22B1030A1002108A300A9144121DA21A8
:1004A000A10B4B2AA9154121851D522A27201F3057
:1004B000A400A91530211020851D612AA40B592AFA
:1004C000C72B1030A1002108A300A9143021DA2184
:1004D000A10B632AA9153021851D6A2A27201F3008
:1004E000A400A9151F211020851D792AA40B712AAB
:1004F000C92B1030A1002108A300A9141F21DA2163
:10050000A10B7B2AA9151F21851D822A27201F30B8
:10051000A400A9150E211020851D912AA40B892A5B
:10052000CB2B1030A1002108A300A9140E21DA2141
:10053000A10B932AA9150E21851D9A2A27201F3069
:10054000A400A915FD201020851DA92AA40BA12A0D
:10055000D32B1030A1002108A300A914FD20DA211B
:10056000A10BAB2AA915FD20851DB22A27201F301B
:10057000A400A915EC201020851DC12AA40BB92ABE
:10058000D82B1030A1002108A300A914EC20DA21F7
:10059000A10BC32AA915EC20851DCA2A27201F30CC
:1005A000A400A915DB201020851DD92AA40BD12A6F
:1005B000DA2B1030A1002108A300A914DB20DA21D6
:1005C000A10BDB2AA915DB20851DE22A27201F307D
:1005D000A400A915CA201020851DF12AA40BE92A20
:1005E000DC2B1030A1002108A300A914CA20DA21B5
:1005F000A10BF32AA915CA20851DFA2A27201F302E
:10060000A400A915B9201020851D092BA40B012BCE
:10061000E42B1030A1002108A300A914B920DA218D
:10062000A10B0B2BA915B920851D122B27201F30DC
:10063000A400A915A8201020851D212BA40B192B7F
:10064000E92B1030A1002108A300A914A820DA2169
:10065000A10B232BA915A820851D2A2B27201F308D
:10066000A400A91597201020851D392BA40B312B30
:10067000EB2B1030A1002108A300A9149720DA2148
:10068000A10B3B2BA9159720851D422B27201F303E
:10069000A400A91586201020851D512BA40B492BE1
:1006A000ED2B1030A1002108A300A9148620DA2127
:1006B000A10B532BA9158620851D5A2B27201F30EF
:1006C000A400A91575201020851D692BA40B612B92
:1006D000F42B1030A1002108A300A9147520DA2101
:1006E000A10B6B2BA9157520851D722B27201F30A0
:1006F000A400A91564201020851D812BA40B792B43
:10070000962B1030A1002108A300A9146420DA213F
:10071000A10B832BA9156420851D8A2B2720A917DF
:10072000552027202917B8212720E529A9012720AE
:10073000291655202720291655202720291655200F
:10074000272027202916962127202916A721272090
:100750002916B82127202916972027202916C921D4
:1007600027202720E5292720291763212720292A48
:100770002720292A2720291741212720291730211E
:100780002720712A2720291730212720712A272086
:10079000712A2720892A27202917FD202720291799
:1007A000EC202720D12A2720A917EC202720D12AA6
:1007B0002720D12A2720E92A27202917B9202720F6
:1007C0002917A8202720312B27202917A8202720E8
:1007D000312B2720312B2720492B27202917752043
:1007E000272029176420962B272029176420962B71
:0407F000FF23900053
:02400E00D43F9D
:00000001FF
